:020000000F28C7
:10000800FE00030EF1000408F2000A08F300831250
:100018007F08F4008D2CD22CEF28F628FD2804291F
:100028000B2912291929202927292E2935293C2964
:1000380043294A29512958295F2966296D29742994
:100048007B2982298929902997299E29A529AC29C4
:10005800B329BA29C129432848284D287A287A285B
:100068007A287A287A28522857285C28612866280E
:100078006B28702875288312A100A00180285330AE
:10008800A4008430A5008B284730A4008430A50044
:100098008B284E30A4008430A5008B28F030A400B3
:1000A8008330A5008B281030A4008430A5008B284D
:1000B8007B30A4008330A5008B284730A400833010
:1000C800A5008B282E30A4008430A5008B28CF30C3
:1000D800A4008330A5008B281230A4008330A5002B
:1000E8008B28AD30A4008330A5008B284E30A400A7
:1000F8008430A5008B288B28210884001030040246
:1001080003187A2800308A002F3004078200250857
:10011800FF00240884000023F5007508A2000130C0
:10012800A4070318A50A0030A507A9010F2A250866
:10013800FF00240884000023F5007508A30001309F
:10014800A4070318A50A0030A507CD284030F500FC
:100158007508A600EA282030F5007508A600EA28E8
:100168001030F5007508A600EA280830F500750873
:10017800A600EA280430F5007508A600EA2802302F
:10018800F5007508A600EA28A6010314A60DEA28BA
:10019800EA282308E039F500F6017608003A031941
:1001A800D628C8287508203A0319AA28603A0319DE
:1001B800AF28203A0319B428E03A0319B928203A9D
:1001C8000319BE28603A0319C328C8282608F50071
:1001D8007508A800CF29EE308316920007308312E5
:1001E8009200E629E13083169200073083129200CC
:1001F800E629D43083169200073083129200E6294C
:10020800C83083169200073083129200E629BD3069
:1002180083169200073083129200E629B2308316C3
:100228009200073083129200E629A83083169200C4
:10023800073083129200E6299E3083169200073019
:1002480083129200E62996308316920007308312B3
:100258009200E6298D3083169200073083129200AF
:10026800E629853083169200073083129200E6292A
:100278007E3083169200073083129200E62976308A
:1002880083169200073083129200E6297030831695
:100298009200073083129200E62969308316920093
:1002A800073083129200E6296330831692000730E4
:1002B80083129200E6295E3083169200073083127B
:1002C8009200E62959308316920007308312920073
:1002D800E629543083169200073083129200E629EB
:1002E8004F3083169200073083129200E6294A3075
:1002F80083169200073083129200E629463083164F
:100308009200073083129200E62942308316920049
:10031800073083129200E629FC30831692000530DC
:1003280083129200E629EE3083169200053083127C
:100338009200E629E130831692000530831292007C
:10034800E629D43083169200053083129200E629FC
:10035800C83083169200053083129200E629BD301A
:1003680083169200053083129200E629B230831674
:100378009200053083129200E629A8308316920075
:10038800053083129200E629831692010730831202
:100398009200E629E62923081F39F500F6017608B8
:1003A800003A0319D829C8297508FF3E031CC82933
:1003B80084001F3004020318C82900308A00103056
:1003C800040782002208F5007508A7007D30810027
:1003D8008B1683161208F5000310750C8312930010
:1003E8000C3095008B17FA296400FA298312A908A2
:1003F800031DFF29002A052A0519032A042AF829BA
:10040800052A8B139501A90105190B2A0C2A0F2A15
:100418001A2A1A2A0F2A2508FF0024088400002314
:0E0428000038031D182A192A9B281A2A0800DA
:10060000FF1B0A2B83137F1883170008840A031922
:10061000FF0A08007F087F398A000408840A03194A
:10062000FF0A82002634A6348634A8346A34603443
:10063000AA348A34A83486348334A33460348634AC
:10064000A8348A34AD348D34AD348F34AF348D3426
:10065000AD3468346034A0348D34AA348D34AD3474
:100660008D34AD348E34A0348E34AE3491348F3426
:10067000AF346A348034A8348A34AD348D34AD3428
:100680008A34AA348834A8348634A6340034263414
:1006900082348234A23447344E348B34AA348934C1
:1006A00053346E348B34AA34893453346E348B34DF
:1006B000AA348B34493482348234A23447344E34E1
:1006C0008B34AA34893453346E348B34AA3489344D
:1006D00053346E348B34AA348B3449346234A234AC
:1006E00044348E348B348A3489348734A734893443
:1006F000AA346934003430346D348D34AB34AD34C5
:10070000AF34AD34AB34AA348D34AD34AA346D3447
:100710008D34AB34AD34AA34A834A534A63448346F
:10072000A834A634A534A334A534A634A834AA34F6
:1007300068346834A834AA34AB34AA34A834A63454
:10074000A534A334A534A33481348134A134A33433
:100750008534863463344834003413348434A53407
:10076000603480348734A834603480348434A534D1
:10077000A034C0348734A834A034C0348D348B34D2
:10078000C0348534A834A034C0348B344A34A03407
:10079000C034AA3488348534A33485340034113409
:1007A00079347934763477349634773474346034E9
:1007B00079347934763497349634803474346034B0
:1007C00071347134743472349134723499348D3498
:1007D0008F347134913491348034913474340034D2
:1007E0002334913491349134913491349134A5343B
:1007F000AA34AD34B1349034903490349034903481
:100800009034A634AA34AD34B0346F348D348A3485
:100810008D346D344A34CA34CD34D13496340034F6
:10082000263468348A34AA34A834A034A8348D34E9
:100830008834863468348F34AF34A834A034A83474
:1008400090348F348A3488348F349434A834A63466
:10085000A034A63483348A344834003420349534A8
:10086000913495349A34763460349334903493349C
:100870009734753493349134603491348E347334B6
:100880006E346034933491347534733400341034DE
:10089000CD34CE34CF34CE34CD3400341034813422
:1008A0008034813400341034D93400340830F500F9
:1008B0007508F700F801812C5E2C640083128518FE
:1008C000622C632C5D2C051C662C672C6D2C780823
:1008D0000138F5007508F8006D2C7708031D712CA0
:1008E0007A2C7808F5007507F6007608F8007A2C5F
:1008F0007A2C64008312851C7E2C7F2C792C812C11
:10090000812C0130F7027708FF3A031D882C892CCF
:100910005E2C8A2C78088C2C08000B117D3081000D
:100920000130A802031D952C962CA52C2608F0005A
:100930007008A8000130A702031D9F2CA02CA52C35
:10094000A9010314A90DA52CA52C7408FF00730898
:100950008A0072088400710E8300FE0E7E0E09006C
:100960008B01073083129900831691018312950140
:1009700007308316850007308312850083168701B0
:1009800083128701823083168100C62C83120519D9
:10099000CA2CCB2CCE2C56243F20CE2C6400C62C47
:1009A000C62C0F28A601A701A801A9018301B02C1C
:02400E00C9F3F4
:00000001FF
